:100000003BC07BC154C053C052C051C050C04FC050
:100010004EC04DC04CC04BC04AC049C048C047C08C
:1000200046C045C044C00902120001010080190900
:10003000040000000000000012011001FF00000891
:10004000C016DC050201010200010E035500530039
:1000500042006100730070001C0377007700770096
:100060002E00660069007300630068006C002E00BB
:10007000640065000403090411241FBECFE5D4E029
:10008000DEBFCDBF10E0A0E6B0E0E0E1FEE002C0E0
:1000900005900D92A236B107D9F710E0A2E6B0E0C4
:1000A00001C01D92A33AB107E1F795D6B0C6A8CF1B
:1000B0001F93CF93DF936091870016160CF5809104
:1000C0008400C7E9D0E0C81BD109635020E010E8E4
:1000D000809183008D3209F44CC08091620087FDCD
:1000E00009C0CE01B7D52FEF821709F470C0811176
:1000F00020E010E0109362002093610010928700CE
:100100008091600084FF27C0809161008F3F19F1CA
:10011000682F893008F050C0861B809361001BE473
:100120008091620080FD13EC8F5F80936200A8E7EE
:10013000B0E087FD56C0662309F04EC060E070E075
:10014000C62F6930D8F19EE18FEF80936100109344
:100150007700909360009AE086B3837011F4915019
:10016000D9F7992309F0A1C0909388009093820059
:100170009CC08AE580936000683009F0BBCF88811D
:10018000807609F048C040E850E0209380008981E3
:10019000882309F04CC02093810022E05093860010
:1001A000409385008F81882309F0A4CF8E81821728
:1001B00008F0A0CF282F9ECF68E0AECF88E790E070
:1001C00098D09C2F9C5FC83008F0C1CFBDCF8EE186
:1001D0008093600010E08ECFCD01EFD4682F772799
:1001E000AFCFE0918500F091860086FF0DC0962F7D
:1001F00003C084918D9331969150D8F7F093860087
:10020000E093850077279CCF962F02C081918D9334
:100210009150E0F7F3CFCE01A0D3282F8F3F09F004
:10022000C1CF888187FF65CF2E8110E063CF8530F5
:1002300059F0863069F08830D9F08930E9F08A3099
:1002400009F0B0CF21E0AACF8A8180938800AACF9D
:1002500010EC8B818130A1F08230F9F0833009F00D
:10026000A1CF8A81882381F444E750E024E096CF2F
:100270004AE850E021E092CF8A8180938A0092CFB1
:1002800048E350E022E18ACF813059F0823009F012
:1002900089CF4AE450E02EE081CF46E250E022E1EF
:1002A0007DCF48E550E02CE179CFDF91CF911F91D0
:1002B000089585B7836085BF8BB780648BBF089531
:1002C000A82FB92F8FEF9FEF41E050EA615070F0F7
:1002D0002D9138E0722F782796958795269570FF97
:1002E00002C0842795273A95A9F7F0CF809590957D
:1002F0000895E6DF8D939D930895CF93CFB7CF9365
:10030000B09BFECFB09B09C0B09B07C0B09B05C09F
:10031000B09B03C0B09B01C09EC0DF93C09184001E
:10032000DD27C557DF4FB09B02C0DF91EBCF2F9386
:100330000F931F9306B32FEF00FB20F94F933F93CA
:1003400016B34FEF012700FB21F93BE031C04E7F90
:10035000012F16B3216028C0102F4D7F22600000AE
:1003600006B329C04B7F2460012F000016B32BC0B9
:1003700016B3477F28602AC04F7E06B320612CC089
:100380004F7D16B320622FC04F7B06B3206432C06E
:10039000422706B349934FEF0000102710FB20F9C6
:1003A00016B31370A9F1297F91F2012700FB21F9FF
:1003B00006B3237F89F23150F0F1102710FB22F9A8
:1003C00016B3277E79F2012700FB23F92F7C81F2F7
:1003D00006B3102710FB24F92F7971F200C016B371
:1003E000012700FB25F92F7359F200C006B310272F
:1003F00010FB26F9223040F200C016B3012700FBA3
:1004000027F9243028F64F77206816B30000F9CF7B
:100410003B503195333010E41ABFB8F0C31BD040C5
:100420000881033C41F10B3431F11981412F1F77D1
:1004300020918200121731F4093691F10D3279F0D2
:10044000013E69F02227209389003F914F911F912F
:100450000F912F91DF91CF91CFBFCF91189500933E
:1004600089003F914F911F910F912F91DF91CAB752
:10047000C6FD46CFF0CF00918900002331F31091E3
:100480008700112349F534304AF1309387000093F7
:100490008300109184003BE0311B309384001EC028
:1004A000009187000130C4F40AE53091600034FD0A
:1004B00017C000936000C7E7D0E016C0052710E022
:1004C00008BB1FC0052722C0052727C005272CC051
:1004D000052710E008BB33C04AE503C042ED01C068
:1004E000432FC4E1D0E032E017B31360C09A08B3E1
:1004F00017BB5F9353E020E820FF052708BB279533
:1005000017951C3FD8F620FF0527279508BB1795A0
:100510001C3FC0F620FF05272795179508BB1C3FF9
:1005200098F620FF0527279517951C3F08BB70F606
:1005300000C0499120FF052708BB279517951C3F50
:1005400038F620FF0527279508BB17951C3F38F57F
:1005500020FF05272795179508BB1C3F10F520FFA6
:100560000527279517951C3F08BBE8F4242F3A95DB
:1005700019F60C7F5F9108BB00C010918800C6512E
:10058000D04011F01093820010E41ABF016017B33D
:100590001C7F402F4C7F08BB17BB48BB56CF05279D
:1005A000D3CF0527D8CF0527DDCFA398AB9A00007E
:1005B00000009B9904C082E58DB91EB80895A29AE7
:1005C000AA98000000009B9B07C082E58DB981E0DE
:1005D0008EB9A298AA9A089583E58DB91EB8A298FB
:1005E000AA9A0895882339F487E293E09093A200B1
:1005F0008093A100089584E493E09093A2008093F7
:10060000A100089592B782B7891B8C30E0F308955A
:10061000C49AA59AAD9887B38C6287BBC298C598D7
:10062000F1DFC29AEFDFC2988091A1009091A20001
:100630008454934009F00895B8DF089587B3837D0B
:1006400087BB88B3837D88BBA5981DB808950F9399
:100650001F93CF93C82F00E017E00CC0C398CC0FB6
:10066000000FB4990F5FCEDFC59ACCDFC59811504B
:1006700017FD04C0C7FFF2CFC39AF1CF802F99278F
:10068000CF911F910F9108958FB9779BFECF8FB1B6
:10069000992708951F93CF93CFE103C0C150CF3F57
:1006A00051F1E091A100F091A2008CEA0995E0914E
:1006B000A100F091A20083E50995E091A100F091DD
:1006C000A20080E00995182FE091A100F091A2000E
:1006D00080E00995133591F01DB8C59A93DFC59850
:1006E00091DF8091A1009091A20084549340B1F6D3
:1006F0005CDFC150B0F681E090E002C080E090E0A5
:10070000CF911F910895EF92FF920F931F937B015A
:100710008C01862F8170880F880F880FE091A100CF
:10072000F091A20080620995D801C70129E0B69531
:10073000A795979587952A95D1F7E091A100F0911B
:10074000A200099516950795F794E794E091A1000A
:10075000F091A2008E2D0995E091A100F091A200E8
:1007600080E0099599271F910F91FF90EF900895D0
:10077000CF92DF92EF92FF921F93CF936B017C0198
:10078000C42F122F862F8170880F880F880FE09159
:10079000A100F091A20080640995D701C60149E04B
:1007A000B695A795979587954A95D1F7E091A100C1
:1007B000F091A2000995D701C601B695A795979526
:1007C0008795E091A100F091A2000995E091A10028
:1007D000F091A2008C2F09951123B1F0CF3791F041
:1007E0001EE1C2B7C701B6018EDF8F3769F482B749
:1007F0008C1B8D3310F0C2B71150112399F781E093
:1008000090E004C08FE09CD080E090E0CF911F91F9
:10081000FF90EF90DF90CF900895CF92DF92EF920C
:10082000FF921F93CF936B017C01142FE091A100E5
:10083000F091A2008CE40995D701C60169E0B69554
:10084000A795979587956A95D1F7E091A100F091CA
:10085000A2000995D701C601B695A79597958795EA
:10086000E091A100F091A2000995E091A100F09122
:10087000A20080E009951F3F91F01EE1C2B7C701B9
:10088000B60141DF8F3F69F482B78C1B8D3310F0C6
:10089000C2B71150112399F781E090E004C08FE0B6
:1008A0004FD080E090E0CF911F91FF90EF90DF90CC
:1008B000CF9008950F931F938C01E091A100F091C8
:1008C000A20080EA0995812F9927E091A100F0917B
:1008D000A2000995E091A100F091A200802F099556
:1008E000E091A100F091A20080E0099599271F9165
:1008F0000F910895FF920F931F938C01F62EE091B4
:10090000A100F091A20080EC0995812F9927E09138
:10091000A100F091A2000995E091A100F091A20040
:10092000802F0995E091A100F091A2008F2D0995EB
:100930008EE106D080E090E01F910F91FF90089526
:10094000382F20E0231740F492B782B7891B8C33ED
:10095000E0F32F5F2317C0F308951F93CF93DF9326
:10096000EC0110E089818130B9F0823009F49FC038
:10097000833009F49FC08430B9F0873009F471C026
:10098000853009F4FAC08630C1F1883009F4C9C055
:10099000893009F006C1F6C09A9B812F23DE1092A0
:1009A000660036DEA998FDC0809166008823A1F418
:1009B0008B819927982F88272A813327822B932B85
:1009C000AA2797FDA095BA2F80936F00909370008F
:1009D000A0937100B09372008F819927982F882778
:1009E0002E813327822B932B909364008093630096
:1009F00082E0809365001FEFD4C080916600882359
:100A000009F47AC08C81482F552750937400409385
:100A100073002D812F70209375008D819927807F21
:100A2000907082959295907F9827807F9827840F69
:100A3000951F909374008093730020FF04C08091F1
:100A40007300809376008F819927982F88272E81B5
:100A50003327822B932B909364008093630081E073
:100A6000C8CF809166008823A1F48B819927982FA5
:100A700088272A813327822B932BAA2797FDA095BD
:100A8000BA2F80936F0090937000A0937100B09381
:100A900072008F819927982F88272E813327822BE8
:100AA000932B909364008093630083E0A2CFC6DD14
:100AB000A99A77C0E091A100F091A2008A810995DE
:100AC00080936700E091A100F091A2008B810995CD
:100AD00080936800E091A100F091A2008C810995BB
:100AE00080936900E091A100F091A2008D810995A9
:100AF00080936A0014E055C08B819927982F88272E
:100B00002A813327822B932BAA2797FDA095BA2FF2
:100B100080936F0090937000A0937100B093720067
:100B200071CF809166008823A1F48B819927982F3B
:100B300088272A813327822B932BAA2797FDA095FC
:100B4000BA2F80936F0090937000A0937100B093C0
:100B500072001092740010927300109375008F81D0
:100B60009927982F88272E813327822B932B9093B8
:100B700064008093630084E03CCF8CDD8093670049
:100B800011E00FC081E0809366008A819B81AC8177
:100B9000BD8180936F0090937000A0937100B0931B
:100BA000720087E690E09093860080938500812F05
:100BB0009927DF91CF911F910895EF92FF921F9394
:100BC000CF937C01162F90916500892F825082303F
:100BD000D0F5C0E0C61710F12FC080916F00909142
:100BE000700068DEF701EC0FF11D808380916F00CB
:100BF00090917000A0917100B09172000196A11DBA
:100C0000B11D80936F0090937000A0937100B0931A
:100C10007200CF5FC11780F4909165009230E9F6C1
:100C200080916F0090917000A0917100B09172005E
:100C3000BC01CD0168DDD6CF183010F410926500EC
:100C4000812F992702C08FEF90E0CF911F91FF90E5
:100C5000EF900895BF92CF92DF92EF92FF920F93A1
:100C60001F93CF93DF936C01062FBB242091650067
:100C7000213019F0243009F0A2C010E0101708F05C
:100C80009BC0213009F05FC0809173009091740087
:100C9000892B09F064C0C12FDD27FE01EC0DFD1D7D
:100CA00080916F0090917000A0917100B0917200DE
:100CB0004081BC01CD015CDD8091630090916400B6
:100CC00001979093640080936300892B09F510923B
:100CD00065008091750081FF19C080917600282FF2
:100CE000332780917300909174002817390771F0B1
:100CF000CC0DDD1D80916F0090917000A09171006E
:100D0000B09172004881BC01CD0187DDC1E0BC2EED
:100D100080916F0090917000A0917100B09172006D
:100D20000196A11DB11D80936F0090937000A09358
:100D30007100B09372001F5F1017F0F520916500ED
:100D4000213009F4A1CFC12FDD27FE01EC0DFD1DDF
:100D5000608180916F0090917000CCDDADCFC12F8C
:100D6000DD277E01EC0CFD1C80916F0090917000DE
:100D7000A0917100B091720020E0F7014081BC01A8
:100D8000CD01F6DC80917600815080937600882337
:100D900009F092CF80916F0090917000A091710046
:100DA000B0917200F7014081BC01CD0136DD809128
:100DB00073008093760080CF8B2D992702C08FEF30
:100DC00090E0DF91CF911F910F91FF90EF90DF9016
:100DD000CF90BF900895CFE5D4E0DEBFCDBF12BA6B
:100DE00018BA8BEF81BB8FEF87BB90E09150F1F782
:100DF0008150D9F787BB93E094BB8EEF85BB93BF3F
:100E000081E0F0DB56DA789453D952D9FDCFFFCF89
:020E10005AFF87
:00000001FF
